:020000040000FA
:020000000528D1
:040002000034003492
:0800080009008C0123008C01AA
:1000100021006A30990021000F308C0020008B01F4
:100020008C01AE01A201A301A401A501A601A701B3
:10003000A001A1010C192D280C192F280030200235
:1000400003191A280830200203183328A10A0C309B
:10005000210203193628A0011A2800000000000020
:100060000000A00A1A28A001A1011A28A001A101DC
:100070000C1946280C19482800302002031938288A
:100080000830200203184C28A00138280000000086
:1000900000000000A00A382896019701A001A101E4
:1000A000A1150C1964280C196628003020020319C8
:1000B00051280830200203186A28A20D2214A10B2F
:1000C00062286E28A00151280000000000000000F6
:1000D000A00A5128A20D2210A10B6228A001A101A3
:1000E0000C197E280C198028003020020319702872
:1000F0000830200203188428A00112280000000004
:1001000000000000A00A7028A001A101A1150C198F
:100110009A280C199C2800302002031987280830DF
:1001200020020318A028A30D2314A10B9828A428AB
:10013000A00187280000000000000000A00A872816
:10014000A30D2310A10B9828A001A1010C19B4281C
:100150000C19B628003020020319A6280830200206
:100160000318BA28A00112280000000000000000B7
:10017000A00AA628A001A101A1150C19D0280C19CC
:10018000D228003020020319BD28083020020318AD
:10019000D628A40D2414A10BCE28DA28A001BD284E
:1001A0000000000000000000A00ABD28A40D2410DB
:1001B000A10BCE28A001A1010C19EA280C19EC28EA
:1001C000003020020319DC28083020020318F02830
:1001D000A0017C290000000000000000A00ADC282B
:1001E000A001A101A1150C1906290C19082900303C
:1001F00020020319F3280830200203180C29A50D4A
:100200002514A10B04291029A001F32800000000E7
:1002100000000000A00AF328A50D2510A10B042959
:10022000A001A1010C1920290C192229003020025B
:10023000031912290830200203182629A0017C295D
:100240000000000000000000A00A1229A001A10186
:10025000A1150C193C290C193E2900302002031964
:1002600029290830200203184229A60D2614A10BC3
:100270003A294629A00129290000000000000000B9
:10028000A00A2929A60D2610A10B3A29A001A10137
:100290000C1956290C195829003020020319482935
:1002A0000830200203185C29A0017C29000000000E
:1002B00000000000A00A4829A001A101A1150C1905
:1002C00072290C1974290030200203195F290830A3
:1002D000200203187829A70D2714A10B70297C2967
:1002E000A0015F290000000000000000A00A5F29B3
:1002F000A70D2710A10B7029220823062406250626
:1003000026062706031D122800306F22A90001309F
:100310006F22AA0003306F22AB002308FE39A80029
:1003200022082906031DAE2928082A06031DAE2926
:100330002318A4298C120000C12200000C162B1CCB
:100340001228B1220C1212280C120000C122000047
:100350008C162B1C1228B1228C1212282209031D84
:10036000B329AE01122822080319582AA21BBE295C
:100370007039703A0319CD29AE011228AE01122846
:10038000EC302302031D12280730240603197A2AB1
:100390002508B00024085F2210282E1CBC29A508BF
:1003A0000319152A2208783A0319DF292208743A1A
:1003B0000319FD2922087C3A0319052A1228241A58
:1003C000122823086F22AF00F021AF05A41DEC29ED
:1003D0002F08031D992212282F0803199922122889
:1003E00001308A00240807398207013402340434BA
:1003F0000834103420344034803423086F2224021F
:10040000031D1228AE019922122807302306031D6E
:100410000E2A08302406031D962A7E2A2408B000DE
:1004200023085F22AE0199221228221D262AA21833
:100430001228221C432A1C2A2308AC00AC030310F8
:10044000AC0D0310AC0DAE1499221228AE1C12286C
:10045000220803392C07AD0007302D060319752A31
:10046000A21D3A2A2308B0002D085F22AD01AE017B
:10047000992212282D086F222302031D1228AD0194
:10048000AE0199221228AE1C1228A21D4F2A230861
:10049000B0001C305F22AC01AE01992212281C3042
:1004A0006F222302031D1228AC01AE0199221228EB
:1004B00022082306031D12282E148C011228230063
:1004C0009100200030082300930015155530960048
:1004D000AA309600951495186B2A20000800230076
:1004E0009100151413082000080008302306031D8E
:1004F000962A7E2A08302506031D12288100F8005E
:100500001E0000000000000020001D008130B0002F
:1005100000305F22F830B00001305F220A30B000B6
:1005200002305F220130B00003305F22AC012E1098
:1005300010288C120C16A922A922A922A922A922CC
:10054000A9220C12080000000230B100B10BA62A4B
:1005500008004730B200A322AD2AB20BAB2A00003C
:10056000080002306F22B6000A30B400C830B5006F
:1005700000000000B50BB82AB40BB62AB60BB42A9B
:1005800008001430B50000000000B50BC32A0800B5
:020000040001F9
:02000E00A40943
:02001000FF1CD3
:10E000008100F8000A0001000000000009009C00E7
:00000001FF
